S01A000064656D6F70726F675F73746D3332673037312E7372656396
S31508002000F00400209D3F0008272E00080B36000824
S3150800201000000000000000000000000000000000B2
S315080020200000000000000000000000000F36000855
S315080020300000000000000000BF3600086B3D0008E5
S315080020408B3D0008373E00087B3F0008873F0008A5
S31508002050E53F0008E73F0008E93F0008EB3F0008B6
S31508002060ED3F0008EF3F0008F13F0008F33F000886
S31508002070F53F0008F73F0008F93F0008FB3F000856
S31508002080FD3F0008FF3F0008014000080340000824
S315080020900540000807400008094000080B400008F2
S315080020A00D4000080F4000081140000813400008C2
S315080020B0154000081740000819400008EE11AA55F7
S315080020C038B5040015D025007C356868002804D189
S315080020D000202870200000F0A5FE242068602068F3
S315080020E00168012291430160200000F0CBF8012825
S315080020F001D1012032BDA06A002802D0200000F0DC
S31508002100B3FD20684168084A0A4042602068816831
S315080021102A22914381602068016801220A430260ED
S31508002120200000F006FE32BDFFB7FFFFF8B584B009
S3150800213007001E007C308068202800D09CE00C0038
S315080021400FD068460280104600280AD080256D0107
S31508002150B868A84207D13869002804D12000C0070A
S3150800216001D5012089E07C20385C012800D183E074
S3150800217001207C217854002039007C31C860222057
S3150800218039007C31886000F04FFE694609885C2278
S31508002190B952694609883A005C325180B968A94241
S315080021A00CD13969002904D135493A005C3291804D
S315080021B027E0FF213A005C32918022E000290CD109
S315080021C03969002904D1FF213A005C32918018E070
S315080021D07F213A005C32918013E02A0491420CD1A7
S315080021E03969002904D17F213A005C32918008E0E0
S315080021F03F213A005C32918003E000213A005C32CC
S31508002200918039005C318988BA68AA4209D13A694D
S31508002210002A06D100222500039602900191140097
S3150800222011E022000025F7E701402170641C07E051
S315080022303868002C406A0199F6D101402980AD1C06
S315080022407088401E70803E005C36708800280BD06F
S3150800225003980090029B00222021380000F098FD88
S315080022600028E5D0032008E038007C302021816072
S3150800227000210170084600E0022005B0F0BD00000C
S31508002280FF010000FEB507000024264620463968EF
S315080022900A683E4B1340BA681A433B6913437A6986
S315080022A01A43FB6913437A6E1A430A6039684A6807
S315080022B0374B1340FA681A434A60B96900913A687D
S315080022C034498A4203D0009D3B6A2B4300939568A4
S315080022D0314B2B40009D1D4395603A68D36A0F2504
S315080022E0AB437D6A1D43D5623A682C4B9A4223D18B
S315080022F02B4B1B689B079B0F5AD0022B2BD059D30D
S31508002300032B59D01023019301258A4200D06FE28E
S315080023101946002909D0022900D17FE0042900D1F5
S31508002320B2E0082900D1E6E01BE101F092F8796AEB
S31508002330002943D129006EE01A4B9A420DD1184B59
S315080023401B680C251D4033D0042D33D0082D02D030
S315080023500C2D31D0D6E70223D5E7134B9A4227D066
S31508002360124B9A4224D08A42CCD10D4B1D68C02309
S315080023701B012B401CD00D0DAB421BD0CD0CAB4224
S31508002380E9D0C0252D01AB4216D0BBE7F369FFCFD4
S31508002390FFCFFFFF00800040FFF4FF110038014027
S315080023A0541002400044004000480040004C0040E1
S315080023B00346A8E70423A6E70823A4E7012901D1D1
S315080023C0022128E0022901D1042124E0032901D1B0
S315080023D0062120E0042901D108211CE0052901D1A4
S315080023E00A2118E0062901D10C2114E0072901D198
S315080023F0102110E0082901D120210CE0092901D17A
S31508002400402108E00A2901D1802104E00B2901D1E5
S31508002410290200E0290001F041F8A3E0786A0028C3
S3150800242001D129002CE0012801D1022128E0022847
S3150800243001D1042124E0032801D1062120E0042843
S3150800244001D108211CE0052801D10A2118E0062837
S3150800245001D10C2114E0072801D1102110E0082829
S3150800246001D120210CE0092801D1402108E00A28E1
S3150800247001D1802104E00B2801D1290200E02900BE
S315080024808C4801F00BF86DE000F096FF796A002998
S3150800249001D129002CE0012901D1022128E00229D5
S315080024A001D1042124E0032901D1062120E00429D1
S315080024B001D108211CE0052901D10A2118E00629C5
S315080024C001D10C2114E0072901D1102110E00829B7
S315080024D001D120210CE0092901D1402108E00A296F
S315080024E001D1802104E00B2901D1290200E029004D
S315080024F000F0D4FF36E0786A002801D129002CE0E4
S31508002500012801D1022128E0022801D1042124E072
S31508002510032801D1062120E0042801D108211CE066
S31508002520052801D10A2118E0062801D10C2114E05A
S31508002530072801D1102110E0082801D120210CE03C
S31508002540092801D1402108E00A2801D1802104E0A8
S315080025500B2801D1290200E02900E80300F09EFFBC
S3150800256000E02E00002800D172E3796800914A0045
S315080025705118884203D300990903814201D22E00DB
S3150800258066E30198002808D002284DD0042800D117
S3150800259092E0082800D1D6E01AE100F05AFF796ADD
S315080025A0002901D129002CE0012901D1022128E0C6
S315080025B0022901D1042124E0032901D1062120E0C2
S315080025C0042901D108211CE0052901D10A2118E0B6
S315080025D0062901D10C2114E0072901D1102110E0A8
S315080025E0082901D120210CE0092901D1402108E060
S315080025F00A2901D1802104E00B2901D1290200E032
S3150800260029007C6800F04AFF0021020E11430002EF
S3150800261002000B006008002180185941220000239F
S3150800262000F093FF0400D4E0786A002801D129005D
S315080026302CE0012801D1022128E0022801D1042139
S3150800264024E0032801D1062120E0042801D108212D
S315080026501CE0052801D10A2118E0062801D10C2121
S3150800266014E0072801D1102110E0082801D1202103
S315080026700CE0092801D1402108E00A2801D180216F
S3150800268004E00B2801D1290200E02900094800F0DE
S3150800269005FF02000023100E0343120200984008AB
S315080026A0002180185941009A002300F04EFF0400CB
S315080026B08FE000BF0024F40000F07EFE796A00294E
S315080026C001D129002CE0012901D1022128E00229A3
S315080026D001D1042124E0032901D1062120E004299F
S315080026E001D108211CE0052901D10A2118E0062993
S315080026F001D10C2114E0072901D1102110E0082985
S3150800270001D120210CE0092901D1402108E00A293C
S3150800271001D1802104E00B2901D1290200E029001A
S315080027207C6800F0BBFE0021020E11430002020085
S315080027300B0060080021801859412200002300F090
S3150800274004FF040045E0786A002801D129002CE03E
S31508002750012801D1022128E0022801D1042124E020
S31508002760032801D1062120E0042801D108211CE014
S31508002770052801D10A2118E0062801D10C2114E008
S31508002780072801D1102110E0082801D120210CE0EA
S31508002790092801D1402108E00A2801D1802104E056
S315080027A00B2801D1290200E02900E80300F076FE93
S315080027B002000023100E034312020098400800216D
S315080027C080185941009A002300F0BFFE040000E07B
S315080027D02E00044820180449884207D23868C46085
S315080027E036E200BF00FDFFFF00FD0F002E002FE2BE
S315080027F0E803F9698142194600D018E1002908D092
S31508002800022946D0042900D182E0082900D1BFE078
S31508002810FCE000F01EFE796A002901D129002CE0AF
S31508002820012901D1022128E0022901D1042124E04D
S31508002830032901D1062120E0042901D108211CE041
S31508002840052901D10A2118E0062901D10C2114E035
S31508002850072901D1102110E0082901D120210CE017
S31508002860092901D1402108E00A2901D1802104E083
S315080028700B2901D1290200E029007C6800F00EFE30
S31508002880400061084018210000F008FE0400A4B2C8
S31508002890BDE0786A002801D129002CE0012801D181
S315080028A0022128E0022801D1042124E0032801D1CD
S315080028B0062120E0042801D108211CE0052801D1C1
S315080028C00A2118E0062801D10C2114E0072801D1B5
S315080028D0102110E0082801D120210CE0092801D197
S315080028E0402108E00A2801D1802104E00B2801D103
S315080028F0290200E029007C68914800F0CFFD4000DD
S3150800290061084018210000F0C9FD0400A4B27EE069
S3150800291000F052FD796A002901D129002CE001292D
S3150800292001D1022128E0022901D1042124E003294A
S3150800293001D1062120E0042901D108211CE005293E
S3150800294001D10A2118E0062901D10C2114E0072932
S3150800295001D1102110E0082901D120210CE0092914
S3150800296001D1402108E00A2901D1802104E00B2980
S3150800297001D1290200E029007C6800F08FFD4000A3
S3150800298061084018210000F089FD0400A4B23EE069
S31508002990796A002901D129002CE0012901D10221F7
S315080029A028E0022901D1042124E0032901D10621C6
S315080029B020E0042901D108211CE0052901D10A21BA
S315080029C018E0062901D10C2114E0072901D11021AC
S315080029D010E0082901D120210CE0092901D1402164
S315080029E008E00A2901D1802104E00B2901D1C10997
S315080029F000E029007C6800F051FD4000610840189D
S31508002A00210000F04BFD0400A4B200E02E0095481A
S31508002A1021001039814208D221000840610849077F
S31508002A20490F01433868C16012E12E0010E1002900
S31508002A3008D0022945D0042900D183E0082900D10D
S31508002A40BFE0FBE000F005FD796A002901D1290005
S31508002A502CE0012901D1022128E0022901D1042113
S31508002A6024E0032901D1062120E0042901D1082107
S31508002A701CE0052901D10A2118E0062901D10C21FB
S31508002A8014E0072901D1102110E0082901D12021DD
S31508002A900CE0092901D1402108E00A2901D1802149
S31508002AA004E00B2901D1290200E029007C6800F026
S31508002AB0F5FC61084018210000F0F0FC0400A4B2FF
S31508002AC0BDE0786A002801D129002CE0012801D14F
S31508002AD0022128E0022801D1042124E0032801D19B
S31508002AE0062120E0042801D108211CE0052801D18F
S31508002AF00A2118E0062801D10C2114E0072801D183
S31508002B00102110E0082801D120210CE0092801D164
S31508002B10402108E00A2801D1802104E00B2801D1D0
S31508002B20290200E029007C68054800F0B7FC610826
S31508002B304018210000F0B2FC0400A4B27FE000BFF8
S31508002B400024F40000F038FC796A002901D1290034
S31508002B502CE0012901D1022128E0022901D1042112
S31508002B6024E0032901D1062120E0042901D1082106
S31508002B701CE0052901D10A2118E0062901D10C21FA
S31508002B8014E0072901D1102110E0082901D12021DC
S31508002B900CE0092901D1402108E00A2901D1802148
S31508002BA004E00B2901D1290200E029007C6800F025
S31508002BB075FC61084018210000F070FC0400A4B2FE
S31508002BC03DE0796A002901D129002CE0012901D1CB
S31508002BD0022128E0022901D1042124E0032901D198
S31508002BE0062120E0042901D108211CE0052901D18C
S31508002BF00A2118E0062901D10C2114E0072901D180
S31508002C00102110E0082901D120210CE0092901D161
S31508002C10402108E00A2901D1802104E00B2901D1CD
S31508002C20C10900E029007C6800F038FC61084018FA
S31508002C30210000F033FC0400A4B200E02E002000BE
S31508002C4010380849884202D23868C46000E02E006D
S31508002C503800683029004180058000214160816084
S31508002C603000FEBDF0FF00002821415CC90706D5EB
S31508002C7001684A68604B1340C26A1A434A602821B1
S31508002C80415C890706D501684A685C4B1340026BAC
S31508002C901A434A602821415C490706D501684A68F3
S31508002CA0574B1340426B1A434A602821415C090777
S31508002CB006D501684A68534B1340826B1A434A602B
S31508002CC02821415CC90606D501688A684E4B13401F
S31508002CD0C26B1A438A602821415C890606D50168B9
S31508002CE08A684A4B1340026C1A438A602821415C61
S31508002CF0490612D501684A68454B1340426C1A4387
S31508002D004A60416C80225203914206D101684A68A2
S31508002D10404B1340826C1A434A602821415C0906DD
S31508002D2006D501684A683C4B1340C06C1843486096
S31508002D307047F8B505002F007C370024FC6000F0CA
S31508002D4073F806002868006800070AD5334800901B
S31508002D503300224680218903280000F019F800284C
S31508002D600ED12868006840070CD52C48009033001F
S31508002D7022468021C903280000F00AF8002801D05D
S31508002D800320F2BD20207860B8603C702046F2BD72
S31508002D90F8B5069E04000D00684602701F002068FC
S31508002DA0C0692840A84201D1012000E000206946F8
S31508002DB0097888421DD10020C0438642EFD000F032
S31508002DC033F8C01B864201D3002EE8D1206801687B
S31508002DD0134A0A4002602068816801229143816093
S31508002DE020007C3020214160816000210170032091
S31508002DF0F2BD0020F2BD0000FFFFFDFFFFFFFEFF52
S31508002E00FFFFFBFFFF7FFFFFFFEFFFFFFFDFFFFF78
S31508002E10FFFFEFFFFFFF9FFFFFFFF7FFFFFFFF012A
S31508002E205FFEFFFF7047FEE701480068704700BF76
S31508002E300000002002480168E020C00108407047F1
S31508002E4008100240FEB5050000D1F9E1B44C287817
S31508002E50C00712D5A16838200840E1688907890F9C
S31508002E60102801D1032901D0082867D120688003DA
S31508002E7003D56868002800D1E2E10220009028689E
S31508002E800221014034D0A16838200840E16889074A
S31508002E90890F102801D1022902D0002800D08AE023
S31508002EA02168490503D5E968002900D1C8E16168A8
S31508002EB0AE4A0A406969090211436160002810D1C7
S31508002EC02068AB490140286908432060A9480121C8
S31508002ED02268D20A5207520F914000F0DFFAA6493B
S31508002EE00860A648006800F065FB002800D0A7E146
S31508002EF0287800070DD5A06838210140182900D088
S31508002F008BE0206E0099014003D0A869002800D103
S31508002F1096E12878400700D40AE10027A0683821FE
S31508002F200140202900D09EE0E06D0099014000D1C3
S31508002F30FEE0A868002800D0FAE081E169688020F0
S31508002F404002814203D121680843206013E0A02291
S31508002F50D202914207D1216882000A432260216881
S31508002F600843206007E02068B749014021602068CF
S31508002F70B649014021608027BF02686800280DD045
S31508002F80FFF752FF06002068384000D075E7FFF7C4
S31508002F904BFF801B6528F6D30320FEBDFFF744FFD1
S31508002FA006002068384000D167E7FFF73DFF801B21
S31508002FB06528F6D3F0E7270DE868002820681CD0B6
S31508002FC06B4901402869084320602068A10D014328
S31508002FD02160FFF729FF06002068384005D1FFF772
S31508002FE023FF801B0328F7D3D6E760685F490140B3
S31508002FF068690002084360607AE7954901402160E4
S31508003000FFF712FF06002068384000D170E7FFF787
S315080030100BFF801B0328F6D3BEE7A8690028206E9D
S3150800302010D0012101432166FFF7FEFE0600206E3F
S315080030300099014000D06CE7FFF7F6FE801B0328D5
S31508003040F5D3A9E7012188432066FFF7EDFE0600C0
S31508003050206E0099014000D15BE7FFF7E5FE801B73
S315080030600328F5D398E780204005E16B014007D196
S31508003070E16B0143E163E16B084001900198012788
S3150800308074480068C00512D472480068A10D01434F
S3150800309070480160FFF7C8FE06006E480068C00564
S315080030A005D4FFF7C1FE801B0328F6D374E7A8688A
S315080030B0012804D1E06D01210143E16511E00528ED
S315080030C0E06D07D104210143E165E06D012101436B
S315080030D0E16506E001218843E065E06D0421884347
S315080030E0E065A86800280DD0FFF79EFE0600E06D93
S315080030F00099014016D1FFF797FE801BAA4988421E
S31508003100F5D349E7FFF790FE0600E06D0099014008
S3150800311008D0FFF789FE801BA3498842F5D33BE711
S3150800312000100240012F03D1E06BA0490140E16382
S31508003130E869002800D185E0A16838220A40102AEB
S3150800314059D08027BF049A49022820683DD10140FA
S315080031502160FFF769FE06002068384010D0FFF7A7
S3150800316063FE801B0328F7D316E700BFFF80FFFF27
S31508003170FFC7FFFF0024F4000C0000200400002015
S31508003180E0688C490140286A0843696A0143A86ACD
S3150800319000020843E96A0143286B0843696B014347
S315080031A0E1602068790801432160E068F90001437D
S315080031B0E160FFF739FE05002068384042D1FFF785
S315080031C033FE401B0328F7D3E6E601402160E0689A
S315080031D003218843E060E068A5490140E160FFF704
S315080031E023FE0500206838402CD0FFF71DFE401B43
S315080031F00328F7D3D0E6012822D0E0688107890F93
S315080032002A6A91421CD1702101406A6A914217D1FB
S31508003210FE21C9010140AA6A1202914210D1F82181
S3150800322089030140EA6A91420AD1E0210905014071
S315080032302A6B914204D1400F4007696B884201D03E
S315080032400120FEBD0020FEBDFFFFFEFFFFFFFBFFC6
S31508003250FFFEFFFF00700040F8B5070065D000913B
S31508003260844800684007400F884218D2814C20687D
S3150800327007218843009901432160FFF7D5FD009D8A
S31508003280060020684007400FA84207D0FFF7CCFD8C
S31508003290801B45498842F4D30320F2BD009539685E
S315080032A0764C022001420CD0490704D5A168E022D9
S315080032B0D2010A43A260A1686F4A0A40B96811435D
S315080032C0A1603978C90732D57968012918D12068EB
S315080032D080032AD5A068072290430143A160FFF71F
S315080032E0A3FD0500A068382101407868C000814226
S315080032F01DD0FFF799FD401B2B498842F2D3CBE737
S31508003300022903D120688001E4D40EE0002903D104
S3150800331020684005DED408E0032903D1226E104058
S31508003320D8D102E0E26D1040D4D10120F2BD009858
S31508003330504909684907490F884218D24D4800681C
S3150800334007218843009901434A480160FFF76CFD4D
S31508003350009D0600474800684007400FA84206D06F
S31508003360FFF762FD801B10498842F3D394E738784B
S31508003370400705D5A06842490140F8680843A0609F
S3150800338000F01AF83F49A268120A1207120F9200B3
S31508003390895CC906C90EC8403B4908603B480068B5
S315080033A000F008F9F2BD000089130000FFFFFFEFE7
S315080033B0FFFFFFFE8C80C11130B5304C3820A16864
S315080033C0014009D101212068C00A4007400F814009
S315080033D02F4800F063F830BDA1680140082901D1E3
S315080033E02C4830BDA168014010291FD1E06880072C
S315080033F0800FE16809094907490F491C7F250328F9
S3150800340007D1244800F04AF8E168090A0D406843E4
S3150800341006E01F4800F042F8E168090A0D406843D3
S31508003420E168490F491C00F039F830BDA168014030
S31508003430202902D18020000230BDA1680840182842
S3150800344002D1FA20C00130BD002030BD0E48006808
S31508003450704710B5FFF7FAFF0400FFF7EBFC0E49BB
S31508003460000B8000085CC006C00EC440200010BDDA
S31508003470FFFFFEEE00200240FFF0FFFF00100240B3
S31508003480FF8FFFFF383E00080C00002004000020D4
S315080034900024F40000127A00303F00080022030AD4
S315080034A08B420BD203098B4219D243088B422ED288
S315080034B0411A00D20146524110467047FF220902BE
S315080034C03FD012068B4205D3121209028B4201D352
S315080034D01212090203098B4219D300E0090AC3092B
S315080034E08B4201D3CB01C01A524183098B4201D3C7
S315080034F08B01C01A524143098B4201D34B01C01AB2
S31508003500524103098B4201D30B01C01A5241C30829
S315080035108B4201D3CB00C01A524183088B4201D398
S315080035208B00C01A524143088B4201D34B00C01A84
S315080035305241884200D3401A5241CFD20146104622
S31508003540704708B500F060F808BD124224D09942C9
S3150800355028D970B500251B4202D00C00002109E0CD
S315080035600024012649186441944200D3A41A7641DE
S31508003570F8D33100012601E0764109D200186441EA
S315080035806D41A41A9D41F7D2A4185D41B619F5D329
S31508003590300022002B0070BD1B42D8D108B500F0C0
S315080035A035F808BD01D19042D3D202000B000021A4
S315080035B00020704770B506000024114DA96800293F
S315080035C01AD0FA208000FFF769FF01000D4800684D
S315080035D0FFF764FF00F057F800280BD1042E07D236
S315080035E0224631000020C04300F049F86E6004E02E
S315080035F0012402E0012400E00124200070BD00BF80
S31508003600000000200C0000207047FEE77047FEE728
S3150800361010B4C20018231340FF249C40E2438901DA
S31508003620C9B2994003000BD5214B0007000F083893
S3150800363080088000181803681A401143016007E0E3
S315080036401C489B089B00C01803681A401143016078
S3150800365010BC704710B5401E80214904884201D32A
S31508003660012010BD144C606003210020C043FFF701
S31508003670CFFF0020A06007202060002010BD80B585
S31508003680FFF7C6FF01BD80B5FFF7E4FF02BD0A4993
S315080036900428086803D1042202430A6070470422FA
S315080036A090430860704780B500F008F801BD000037
S315080036B01CED00E000E400E010E000E07047FEE7E3
S315080036C0FEB507000020050001006A461170754C1A
S315080036D0396889035FD56946487080204005216BA3
S315080036E0014009D1216B01432163216B08400190F8
S315080036F001980120694648706B480068A10D01438E
S3150800370069480160FFF790FB060067480068C00536
S3150800371005D4FFF789FB801B0328F6D30325280069
S315080037202FD1216DC020800008400FD0396B884208
S315080037300CD0216D5D480840216D802252020A4353
S315080037402265216D5A4A0A4022652065C0070CD5B4
S31508003750FFF76AFB0600206D800706D4FFF764FBB7
S31508003760801B54498842F6D30325280006D1206DCC
S315080037704E490140386B0843206504E068460570E9
S3150800378001E06846057068464078012803D1206B39
S315080037904949014021633878C00705D5A06C032143
S315080037A0884379680143A1643878800705D5A06CF9
S315080037B00C218843B9680143A1643878800605D589
S315080037C0A06C3E490140F8680843A0643868800543
S315080037D005D5A06C3A490140B8690843A064386821
S315080037E0400505D5A06C37490140F8690843A0642F
S315080037F03878400605D5A06C334901403869084336
S31508003800A0648020C001396801400DD0A16C8900F0
S3150800381089083A6A0A43A264396A0204914203D1C2
S31508003820216882000A4322603968090305D5A16C1C
S31508003830402291437A6A0A43A26401023A689202D4
S315080038400CD5A26C214B1340BA6A1A43A264BA6A11
S315080038508A4203D122688302134323603A681140DF
S315080038600CD0A16C1A4A0A40F96A1143A164810274
S31508003870FA6A8A4202D12268114321603968090529
S315080038800DD5A16C134A0A4079691143A164796977
S31508003890814204D12068802149020143216068469B
S315080038A00078FEBD0C10024000700040FFFCFFFFD0
S315080038B0FFFFFEFF89130000FFFFFFEFFFF3FFFF87
S315080038C0FFFFF3FFFFFFCFFFFFCFFFFFFFFFBFFFA6
S315080038D0FFFFFFFEFF3FFFFFFFB40A0000230100C2
S315080038E032E0052403E05A4CA142FAD10400AC4068
S315080038F0344300980460574C2568019EF043054000
S315080039005668F60302D52E00019D35432560656885
S3150800391005405668B60302D52E00019D35436560FD
S31508003920803C256805405668F60202D52E00019DA2
S3150800393035432560656828405568AD0202D50500FF
S315080039400198284360605B1C10680400DC4077D04F
S31508003950012425009D4003950540019501980028FE
S31508003960F1D05068022801D0122811D1D808800059
S315080039700D18286A1E00B7001C263E400F27B740C0
S31508003980B8431769BC4637006646BE4006432E62F2
S315080039900D68180040006E46307003203778060020
S315080039A0BE40F74302973E462E40556805406F468F
S315080039B03F78BD4035430D605568012D05D0022D71
S315080039C003D0112D01D0122D11D18E68029D3540DC
S315080039D0D6686F463F78BE402E438E604D68039E7C
S315080039E0B5435668360926409E402E434E60CE683B
S315080039F0029D354096686F463F78BE402E43CE609E
S31508003A005568ED009FD5144D9E08B600AD19009572
S31508003A102E681D00EF0018253D400F27AF40BE4316
S31508003A20A027FF05B94201D1002460E70B4FB94230
S31508003A3000D15CE70A4CA14200D054E7022456E7BD
S31508003A40FFBC7047002A01D08161704781627047C8
S31508003A50000C005080180240601802400004005014
S31508003A600008005080B500F007F800F0B4F800F040
S31508003A702FF900F0B4F8FAE780B500F009F800F07D
S31508003A8049F900F009F800F059F900F019F901BDF3
S31508003A9049484A490860704730B59FB03822002126
S31508003AA004A800F068F910220021684600F063F9BE
S31508003AB03422002112A800F05EF98020800000F070
S31508003AC065F902240494E001079000250895402032
S31508003AD009900B940C9430210D910E90C0020F9012
S31508003AE0000210904806119004A8FFF7ABF90028C9
S31508003AF000D0FEE707200090019402950395214621
S31508003B006846FFF7A9FB002800D0FEE71294149533
S31508003B1012A8FFF7D5FD002800D0FEE71FB030BD7C
S31508003B20F8B586B026480124C1682143C160C1683A
S31508003B3021400091009901682143016001682140F4
S31508003B4000910099022601683143016001683140FD
S31508003B5000910099610482680A4382608068014086
S31508003B6000910098002211460420C043FFF787FD04
S31508003B70002211460120C043FFF781FD00221146AD
S31508003B800020C043FFF77BFD20200190029400250A
S31508003B9003950495A027FF0501A93800FFF79CFEA9
S31508003BA00C200190029603950495059401A9380006
S31508003BB0FFF792FE07B0F0BD0020000808ED00E010
S31508003BC034100240BFF34F8F384839490860BFF3B5
S31508003BD04F8F00BFFDE780B500F009F801BD80B53D
S31508003BE000F01BF801BD80B5FFF7ECFF01BD80B5FD
S31508003BF0304831490160E1210902416000218160B4
S31508003C00C160016181610C224261C1618022120199
S31508003C1002624162FEF754FA01BD38B5274D2C0001
S31508003C2044346078002811D1280000F034F80128BF
S31508003C3030D1287800282DD041282BDA00F091F8C9
S31508003C406060012060700020207031BD681C44212E
S31508003C50695C401800F01FF8012813D14420285C3D
S31508003C60401C207001002A78C9B2914212D1002165
S31508003C7061706978FF290DD1C0B202280AD1FFF711
S31508003C80B2FF31BD00F06DF861686431814201D23E
S31508003C900020607031BD80B501000023012205486F
S31508003CA0FEF744FA401E8041C00F02BD0400FA0523
S31508003CB00CED00E010000020004400409C000020AD
S31508003CC080B500222021A020C005FFF7BBFE01BD5C
S31508003CD038B500F046F805000D4C6068281AFA2138
S31508003CE04900884212D3A020C0052178002906D1B0
S31508003CF0012121700A462021FFF7A4FE05E00021D4
S31508003D0021700A462021FFF79DFE656031BD00003F
S31508003D10E800002010B5002407480168820D0A4310
S31508003D2002602046FFF746FC002801D0012401E086
S31508003D30FFF7F6FE200010BD0020024080B5FFF711
S31508003D4085FBFA218900FFF7A9FBFFF79CFC0420F5
S31508003D50FFF79DFC002211460020C043FFF78FFCA9
S31508003D6001BD80B5FFF760F802BD80B500F034F8F4
S31508003D70FFF799FC01BD10B5040008001100020008
S31508003D80200000F031F8200010BDFEE710B50E4CFB
S31508003D9021680E4A0A4002432260610D884211D109
S31508003DA00B4800684100081840000A49FFF776FBEF
S31508003DB0401C00E0401E6169490503D50028F9D179
S31508003DC0032010BD002010BD00700040FFF9FFFF62
S31508003DD00C00002040420F000248016882688918DA
S31508003DE001607047000000201206130A1A43130CDC
S31508003DF01A4300BF094205D0830705D00270401C4C
S31508003E00491EF9D1704700001300103906D330B4A3
S31508003E101400150010393CC0FCD230BC490700D349
S31508003E200CC000D504C0890002D30280801C00297A
S31508003E3000D502707047FEE7000000000000000091
S31508003E400000000000000000000000000000000064
S31508003E500000000000000000010000000200000051
S31508003E600300000004000000060000000700000030
S31508003E70080000000900000070B40123002413E0C4
S31508003E800168001D194202D04D466D1E49190C6085
S31508003E90091D121F042AFAD20D00960701D50C80B7
S31508003EA0AD1C1A4000D02C700268001D002AE7D10C
S31508003EB070BC704730B401220EE00368C31844682A
S31508003EC00830144202D04D466D1E64191D682560DF
S31508003ED01B1D241D091FF9D10168001D0029ECD1FD
S31508003EE030BC704710B5074979441831064C7C44F4
S31508003EF0163404E0081D0A68891888470100A1429B
S31508003F00F8D110BD08000000280000006DFFFFFF73
S31508003F10E0000000100000200000000099FFFFFFED
S31508003F2010000000A40000000000002000000000AF
S31508003F300000000000000000000000000000000073
S31508003F400100000002000000030000000400000059
S31508003F5000F00DF8002801D0FFF7C4FF00BF00BF2E
S31508003F60002000BF00BFFFF77DFD00F002F801202A
S31508003F70704780B500F002F801BDFEE707463846EF
S31508003F8000F002F8FBE7FEE780B500BF00BF024A73
S31508003F9011001820ABBEFBE726000200034880F399
S31508003FA0088803488047034800470000F0040020BB
S31508003FB0B93F0008D93F000880200005014908607C
S31508003FC07047000008ED00E0000000000400000053
S31508003FD0010000000024F40000BF00BF00BF00BFBE
S31508003FE0FFF7B6FFFEE7FEE7FEE7FEE7FEE7FEE7BA
S31508003FF0FEE7FEE7FEE7FEE7FEE7FEE7FEE7FEE78B
S31508004000FEE7FEE7FEE7FEE7FEE7FEE7FEE7FEE77A
S30F08004010FEE7FEE7FEE7FEE7FEE71F
S70508003FD9DA
